:020000040000FA
:040000006F303A28FB
:08000800A000030EA100831209
:1000100005191028831601178312B23081002B288E
:1000200083160113831203140B190310A80DA90DD5
:10003000AA0DAB0DAC0DAC16FF302C02031D2B2806
:10004000FA302B02031D2B2831152A08AF0029088E
:10005000AE002808AD008B100B11210E8300A00EFE
:04006000200E090065
:0C007400203084008001840A6030040207
:10008000031C3C281230B000972183160C308505E4
:1000900087018312850187010730990000309A009B
:1000A000103083168E008312603083168F00831207
:1000B0000030831691008312C830831681008312AA
:1000C00031309000003083168C00831210308B008A
:1000D000831600309B001C141A088312BC00831680
:1000E00010309B001C141A088312BD00C521831612
:1000F00020309B001C141A088312C2000130C20871
:100100000319C20081018E018F010B118B100B109E
:100110008C018B179A2031199D207921B30B9828D7
:10012000031085190314B90DF03039020319222187
:10013000C6218A2864003210080031110130B7004E
:100140008B132030370783169B001C141A08831268
:10015000A4001030370783169B001C141A08831262
:10016000A300A6000230A6060030370783169B00C6
:100170001C141A088312A200A7000130A7068B17CF
:10018000321CC82822090339A200A309A409A50921
:1001900024082F02031D1C2923082E02031D1C29DD
:1001A00022082D02031D1C2901303702031DDD2802
:1001B0003D18DD283D143E149E2102303702031DF8
:1001C000E628BD18E628BD143E14A72103303702E7
:1001D000031DEF283D19EF283D153E14B0210430D2
:1001E0003702031DF828BD19F828BD153E14B921A2
:1001F00005303702031D01293D1A01293D163E1421
:10020000C12106303702031D0A29BD1A0A29BD166D
:100210003E14C22107303702031D13293D1B132949
:100220003D173E14C32108303702031D1C29BD1B96
:100230001C29BD173E14C421B70A05303702031824
:100240000800A0280130B600B300B400B500B70024
:1002500085018701B1139A20B30B48290310851932
:100260000314B90DF030390203196F29B41F850149
:10027000B41F8701B40B48293708B6080319B60024
:1002800003194629FF3085008700B6039630B40075
:10029000311D2B293111321C52292D090339AD0092
:1002A000AE09AF092F1C2B298E018F010C1C2B29A5
:1002B0000C102E1E2B298B1320303707BB002F0864
:1002C000BA00822110303707BB002E08BA00822105
:1002D00000303707BB002D08BA0082218B1785013B
:1002E0008701B70AB60105303702031C2B29C52147
:1002F00008003E1C08003E101030BB003D08BA004C
:10030000822108008B133A0883161C159A00831269
:100310003B0883169B0055309D00AA309D009C141D
:1003200064009C1890291C1183128B17080001305F
:10033000D500D200EE30D000D10008000130D50049
:10034000D200EE30D000D1000130BD0008000130F5
:10035000D500D200EE30D000D1000230BD00080040
:100360000130D500D200EE30D000D1000430BD0005
:1003700008000130D500D200EE30D000D100BD0120
:100380000800080008000800080008008F0803198A
:1003900008008F01C10B08004208C100D50B0800FE
:1003A0005608D50007303D050319FD29D21BD00A98
:1003B000D21FD0030A305002031CF829D0010930A3
:1003C000D21FD0005203D2007F39031DF829D10A71
:1003D00010305102031CED29D1015022D2006022BD
:1003E000D4007022D600D500D0010930D21FD00031
:1003F0000023850024238700080085018701080069
:1004A00002308A0051083D1C572A883E8200BD1C3C
:1004B0005B2A883E82003D1D5F2A983E8200003400
:1004C00002308A0051083D1C672AA83E8200BD1CEC
:1004D0006B2AB83E82003D1D6F2AB83E8200003470
:1004E00002308A0051083D1C772AC83E8200BD1C9C
:1004F0007B2AD83E82003D1D7F2AE83E82000134DF
:100510000734873407348734033483340334833413
:100520000B3403340F3407340B34033403340734EF
:10053000053487340734253483340334073489344D
:100540000B3403348F3405348B34113403340334C7
:1005500001340134023402340434043408340834DD
:10056000103410342034203440344034803480340B
:10057000083404340234803440348034103402347B
:10058000043410342034013404344034843480344E
:10059000093409340A340A34083408340834083475
:1005A0000834183408341834083418341034083433
:1005B000093429340A341A34283408340834083405
:1005C0000A34383408341A3408345834103448346F
:1005D000293409340A340A342834083408344834B5
:1005E0002834183488341834283418341034083433
:1006000003308A005008541C072B4B3E8200D41C38
:100610000B2B563E8200541D0F2B613E8200D41DD1
:10062000132B6C3E8200541E172B773E8200D41E83
:100630001B2B823E8200541F1F2B8D3E8200D41F35
:10064000232B983E8200003403308A005008541C4B
:100650002B2BA33E8200D41C2F2BAE3E8200541DB8
:10066000332BB93E8200D41D372BC43E8200541E6A
:100670003B2BCF3E8200D41E3F2BDA3E8200541F1C
:10068000432BE53E8200D41F472BF03E820000340E
:0A0696001034203401340234003423
:0A06A000003400340034003400344C
:0406AC0010343034A2
:1006B0003134333433343334333433343334333404
:0E06C2000034003400340034003400340234BC
:0606D0000334233433342F
:0806D800103420340134023417
:0C06E000003410342034013402340034A3
:0206EE001034C6
:1006F0002034013402340034003402340134203414
:020700001034B3
:0C070400103430343134333433343334A7
:080710003134303410340034A0
:06071A00333423340334E4
:0E072000023400340034023403342334333402
:10073000333400343334003433340034333400344D
:04074000333400341A
:0A07460000340034003400340234A3
:0A075000043401342034103408345E
:04075C000034003431
:1007600000340034023406340734273437343F343D
:0E07720008341834383439343D343F343F34C1
:060780003F343F343F341A
:08078800043401342034103464
:0C0790000A3404340134203410340A34DC
:02079E0008341D
:1007A000103420340134063406340134203410343B
:0207B00008340B
:0C07B40008341834383439343F343934F8
:0807C000383418340834003409
:0607CA003F3437342734F0
:0E07D0000734063406340734273437343F34F8
:1007E0003F3400343F3400343F3400343F3400346D
:0407F0003F3400345E
:084000000C00030002000600A1
:02400E00CC33B1
:10420000010078007A007C007E007B0079007F004E
:104210007D007A0078007E007C00FF00FF00FF0038
:104220000000F200F600FA00FE00F200F600FA00CC
:10423000FE00F200F600FA00FE00FF00FF00FF00A3
:10424000010005000500050005000900090009003E
:1042500009000D000D000D000D00FF00FF00FF0024
:10426000FF00FF00FF00FF00FF00FF00FF00FF0056
:10427000FF00FF00FF00FF00FF00FF00FF00FF0046
:10428000FF00FF00FF00FF00FF00FF00FF00FF0036
:10429000FF00FF00FF00FF00FF00FF00FF00FF0026
:1042A000FF00FF00FF00FF00FF00FF00FF00FF0016
:1042B000FF00FF00FF00FF00FF00FF00FF00FF0006
:1042C000FF00FF00FF00FF00FF00FF00FF00FF00F6
:1042D000FF00FF00FF00FF00FF00FF00FF00FF00E6
:1042E000FF00FF00FF00FF00FF00FF00FF00FF00D6
:1042F000FF00FF00FF00FF00FF00FF00FF00DD00E8
:00000001FF
